:107800000C942A3C0C94453C0C94453C0C94453C0F
:107810000C94453C0C94453C0C94453C0C94453CE4
:107820000C94453C0C94453C0C94453C0C94453CD4
:107830000C94453C0C94453C0C94453C0C94453CC4
:107840000C94453C0C94453C0C94453C0C94453CB4
:107850000C94453C11241FBECFE5D8E0DEBFCDBF60
:1078600010E0A0E6B0E0EAE5FFE702C005900D9267
:10787000A036B107D9F711E0A0E6B0E001C01D9233
:10788000A43AB107E1F70C94723F0C94003C0F93BB
:10789000EF93FF933ED0FC01062F35D0FF91EF917F
:1078A0000F9108950F930F921F92EF93FF9331D092
:1078B000FC010B0101E027D0FF91EF911F900F9089
:1078C0000F9108950F930F92EF93FF9322D0FC0135
:1078D00060FD67BFC895802DE395C895902DFF91F9
:1078E000EF910F900F9108950F930F9212D0082EE1
:1078F00009E009D00F900F9108950F930AD001E18C
:1079000002D00F910895E199FECF07BFE895FFFFE0
:10791000000007B700FDFDCF089583E089B9549AB0
:10792000539A08958CB19927089540E050E0481784
:10793000590750F42AE633E000002150304037FF69
:10794000FBCF4F5F5F4FF3CF08958BB199278078BE
:10795000907008955498539808950E94AA3C0C94EE
:10796000000008958CB95E9BFECF5E9A08950E9438
:10797000A53C8823E1F30E94923C803219F481E017
:1079800090E0089585E10E94B23C80E090E0089587
:107990000895EF92FF920F931F93CF93DF937B0194
:1079A000C0E0D0E0C617D70770F48C010E94A53C58
:1079B0008823E1F30E94923CF80181938F01219684
:1079C000CE15DF0598F381E090E0DF91CF911F9114
:1079D0000F91FF90EF90089590E0282F33272138E2
:1079E000310589F02238310524F42038310549F079
:1079F0000DC02238310549F02839310539F493E0BA
:107A000005C092E003C091E001C092E1892F99275F
:107A1000089540E050E06091A0007091A1004617E9
:107A20005707E8F4E2EAF0E08091A2018EBB809172
:107A3000A2019091A301292F33272FBB0196909388
:107A4000A3018093A20180818DBBE29AE19AE19922
:107A5000FECF4F5F5F4F31964617570728F30895C3
:107A60000F931F93CF93DF9300E010E08091A0006D
:107A70009091A10008171907D8F4C2EAD0E08091CC
:107A8000A2019091A301880F991F60E0800F911FC0
:107A90000E94623C8883892F992789830E5F1F4F3C
:107AA00022968091A0009091A1000817190738F341
:107AB000DF91CF911F910F9108958091A000909137
:107AC000A1000097C1F0E2EAF0E0AC018091A201D0
:107AD0008EBB8091A2019091A301292F33272FBB48
:107AE00001969093A3018093A201E09A8DB38193B4
:107AF0004150504059F708950F931F93CF93DF9350
:107B00008C016115710541F0EB01F80181918F0144
:107B10000E94B23C2197C9F781E090E0DF91CF91BC
:107B20001F910F910895EF92FF920F931F93CF93A0
:107B3000DF93C0E0D0E08E017E01CFEFD0E0F09285
:107B4000A301E092A20163E0C8010E94473C219793
:107B500080E490E0E80EF91E00581F4FD7FFEFCFEA
:107B60000E947D3CDF91CF911F910F91FF90EF908C
:107B70000895EF92FF920F931F93CF93DF9300E04E
:107B800010E08091A0009091A1000817190708F05B
:107B900047C0EE24FF24E801CD55DF4FF801EE5534
:107BA000FF4FEE0DFF1D4081888122969927382FC7
:107BB0002227240F311D8091A2019091A301880FEB
:107BC000991FB9018E0D9F1D0E94523C82E090E0EA
:107BD000E80EF91E90E8E916F10400F38091A20185
:107BE0009091A301880F991F63E0800F911F0E945D
:107BF000473C8091A2019091A301880F991F65E0F5
:107C0000800F911F0E94473C0E947D3C00581F4FEF
:107C10008091A0009091A1000817190708F4B9CF2E
:107C2000DF91CF911F910F91FF90EF900895CF9327
:107C3000C0E069E081E090E00E94623C84FF03C004
:107C40008F7E0E94743C0E94A53C8823E1F30E9431
:107C5000923C992782359105DCF4803591050CF032
:107C600054C08134910509F45AC0823491053CF422
:107C70008033910509F449C0C19759F12FC182346D
:107C8000910509F45FC08534910509F45EC026C1F1
:107C90008635910509F4EDC0873591054CF48235A0
:107CA000910509F461C08535910509F465C016C1D7
:107CB0008437910509F4A0C0853791052CF48436EA
:107CC000910509F472C00AC18537910509F4C1C054
:107CD00005C10E94B73C882309F4B5CF84E10E9416
:107CE000B23C81E40E94B23C86E50E94B23C82E54F
:107CF0000E94B23C80E20E94B23C83E50E94B23C0A
:107D000084E50E94B23C8BE406C00E94B73C882305
:107D100009F499CF84E10E94B23C80E1E0C061E0C7
:107D200070E080E690E00E94C93C0E94B73C882346
:107D300009F489CF84E10E94B23C809160000E94E6
:107D4000EC3CE9CF64E170E00AC061E070E080E6FD
:107D500090E00E94C93C809160009927BC0180E6B8
:107D600090E00E94C93CD1CF0E94B73C882309F41F
:107D70006ACF0E94933DCECF62E070E080E690E053
:107D80000E94C93C0E94B73C882309F45CCF209133
:107D90006000809161009927982F8827820F911D9C
:107DA0009093A3018093A201B5CF63E070E080E6D9
:107DB00090E00E94C93C2091610080916000992769
:107DC000982F8827820F911D9093A1008093A00087
:107DD000BC0182EA90E00E94C93C0E94B73C882323
:107DE00009F431CF80916200863419F40E94B93DC4
:107DF00091CF0E94093D8ECF63E070E080E690E075
:107E00000E94C93C20916100809160009927982FC1
:107E10008827820F911D9093A1008093A0000E945B
:107E2000B73C882309F40FCF80916200863419F49F
:107E30000E94303D02C00E945D3D84E10E94B23C40
:107E40006091A0007091A10082EA90E00E947C3DC8
:107E500064CF0E94B73C882309F4F5CE84E10E94E8
:107E6000B23C8EE10E94B23C85E90E94B23C82E0C5
:107E700052CF64E070E080E690E00E94C93C0E942E
:107E8000B73C882309F4DFCE84E10E94B23C8091A4
:107E90006000803531F480916100882361F4C82F3F
:107EA00017C0883531F480916100883061F4C3E0F7
:107EB0000FC0803531F480916100883049F4C2E010
:107EC00007C0883529F480916100882309F4C1E056
:107ED00069E08C2F99270E94623C1DCF85E10E94AA
:107EE000B23CB1CECFE5D8E0DEBFCDBFCEE1F89455
:107EF0008EEF93E00E94A43F843B59F48FEF93E010
:107F00000E94A43F833C29F48DEF93E00E94A43F9C
:107F100081BF0E948D3C0E94923C84E690E00E94CA
:107F2000953C0E94A53C882321F4C150C8BBCC23BA
:107F3000A1F7CC2319F00E94173E02C00E94AD3C6D
:107F400080E090E00C94AC3FE199FECF9FBB8EBBEC
:0A7F5000E09A99278DB30895FFCF42
:040000030000780081
:00000001FF
